:020000040000FA
:1000000007309F00A00183168501860183128501B8
:100010008601E1208517E120851005103F30A500FD
:10002000D120E1204030A500D120B830A500D1205A
:10003000C030A500D120851405107F30A500D12047
:10004000E120851005100030A500D920B930A500A9
:10005000D120851405107F30A500D120851005140E
:100060004030A500D120851005100030A500D92012
:10007000BA30A500D120851405107F30A500D1200D
:10008000851005144030A500D120851005100030E2
:10009000A500D920BB30A500D120851405107F30E4
:1000A000A500D120851005144030A500D120851071
:1000B00005100030A500D920BC30A500D120851442
:1000C00005107F30A500D120851005144030A50013
:1000D000D120851005100030A500D920BD30A50025
:1000E000D120851405107F30A500D120851005147E
:1000F0004030A500D120851005100030A500D92082
:10010000BE30A500D120851405107F30A500D12078
:10011000851005144030A500D12085100510003051
:10012000A500D920BF30A500D120851405107F304F
:10013000A500D120851005144030A500D1208510E0
:1001400005100030A500D9203F30A800BB30A50025
:10015000D120851405104030A500D120851005144C
:100160004130A500D120851005107F30A500D92091
:10017000A80BB7283F30A800BC30A500D1208514BB
:1001800005104030A500D120851005144130A50090
:10019000D12085100510FE30A500D920A80BCD2850
:1001A000D02805112508860085150000851100005E
:1001B000003405152508860085150000851100000E
:1001C0000034FF30EA286430EA283230EA2814305C
:1001D000EA280530A100C730A2000130A300A20B1D
:0C01E000F228A30BEF28A10BEB28003441
:02400E00183D5B
:00000001FF
